:1000000011298030A100FE30AF200130AF207530C3
:10001000A7003030C628A101A117AF00AF08031D0B
:100020001328030114280130AF020310A20CA20C04
:10003000A20CC0302205403EAF07FE30AF202F0893
:10004000AF28A101A117AF00FE30AF202F08AF28C5
:10005000A401AA00AB01A01124080319A0150530C2
:10006000A3002730A900103041200330A900E83058
:100070004120A90164304120A9010A3041202A0809
:100080004828A8002B08A7002A08A600DA2026087E
:10009000A600A3030319A011240803195228230260
:1000A000031859282608031DA011A0195928303E0D
:1000B000AF280800A300240803190C292308AF2047
:1000C000A4035B28AD000611861183160611861164
:1000D0000F30860583122D08A0188C283E30A7000B
:1000E0008030C6203330AC00A0201330A700883009
:1000F000C620A0206430C520A0206430C520223056
:10010000AC00A02028308B200C308B2006308B20B8
:10011000A0142D088C282014AC00201C9A288611CD
:10012000033C031C9F289F200530A700DC30C6201D
:10013000031408002014FE3C0319AD288615201C6A
:10014000201006150F3086052C08F039860406119C
:10015000AC0E2018A0283230C5202D080C29A11B78
:10016000622883178001840AFF3E031DB2280C29F0
:10017000A901A800FF30A807031CA907031C0C292C
:100180000330A700DF30C620BA28A701E83EA6004A
:10019000A709FC30031CCF28A6070318CC28A60704
:1001A0000000A70FCC282618D528A61CD9280000A7
:1001B000D9280800AB01AA011030AC00270DAA0D08
:1001C000AB0D2808AA022908031C290FAB0203184B
:1001D000F0282808AA0729080318290FAB070310DD
:1001E000A60DA70DAC0BDE2826080C291030B00098
:1001F000A701A601AD0CAC0C031C04292808A60716
:1002000029080318290FA707A70CA60CAB0CAA0CEA
:10021000B00BFA282A080C29831383120313000059
:100220000800A00107309F00E03083168500FF30F2
:10023000860081138312850186012030840060309E
:10024000B220A03084005030B22020308400303002
:10025000B120C830B82001207730622062206220AF
:100260002E3062207030622069306220633062205C
:100270006230622061306220733062206930622017
:10028000633062202E3062206E3062206C3062203B
:100290000B30A900B830B92001204430622043302F
:1002A00062204630622032306220303062204E3090
:1002B00062204C3062204430622020306220622074
:1002C000563062202D306220323062200730A90083
:1002D000D030B92001204C306220443062205230AE
:1002E00062202030622061306220663062207230ED
:1002F00062206530622067306220653062206C3099
:100300006220653062206E30622086188D29851F3C
:100310008B2905148C290510852901205330622072
:1003200069306220673062206E3062206130622066
:1003300062206C306220203062207A3062206F3080
:100340006220653062206B306220653062206E3042
:10035000622036140512831605128312442AC30143
:100360003C03A500C90149082502031CC829EB214B
:10037000B61CC6294308A6004908A200A601A20A85
:100380000314A60DA20BC1292608C304C90FB32963
:10039000B2014308B100B20CB10CB20CB10CB20CFA
:1003A000B10CB20CB10C0F30B2053208AD003108FF
:1003B000AC00A9010A30A800F620B1002B08B20059
:1003C000B4014308B3000F30B3050030B405310861
:1003D0003307C3000800BA01B9010618002A01302A
:1003E000B820B90A0319BA0A0B303A02031CFF29D4
:1003F000031DFE29B9303902031CFF29AA2DED295E
:100400009B30B8200618B614061CB610361C242AD9
:10041000AD014408AC00A9011430A800F620B100D9
:100420002B08B2003208A7003108A600A9013A3013
:10043000A800DA20BD008030A1000230A2003D08F3
:100440000D20FF306220372A8030A1000130A20049
:100450003D080D200230A40044082920030136196C
:10046000013EB618013A03193611031D3615C40AA8
:1004700085140130A900F430B9208510A901F030AD
:10048000A8002808B9200800BB01C4013612361A9A
:10049000E92ABA01B901061C5E2AB90A0319BA0A87
:1004A0000130B820AF303A02031C5D2A031D5C2ADC
:1004B000C9303902031C5D2AAA2D4B2ABA01B901A1
:1004C00006189A2AB90A0319BA0A0A30B820361847
:1004D0008E2A39080B3A3A04031D792A8030A1008C
:1004E0000130A2003D080D203530622039306220F5
:1004F0008D2A3908193A3A04031D802A85148D2A59
:1005000039084B3A3A04031D872A85108D2A390889
:10051000FA3A3A04031D8D2AAA2D992A11303A027B
:10052000031C992A031D982A95303902031C992A25
:10053000AA2D602A41303B02031C9F2AAA2DBB0A28
:100540003A08031DA72A65303902031CA82A36166B
:10055000361CE82AAD013B08AC00A9011430A80004
:10056000F620B1002B08B2003208A7003108A6001F
:10057000A9014130A800DA20BD008030A100803000
:1005800021205330622069306220673062206E3053
:1005900062206130622062206C3062202030622054
:1005A0006730622065306220763062206F306220D2
:1005B0006E30622064306220653062206E306220CE
:1005C0008030A1000230A2003D080D20FF306220E3
:1005D000472A361C132B0120493062206E306220DE
:1005E000693062207430622069306220613062209C
:1005F0006C30622069306220733062206530622086
:1006000072306220653062206E3062202E306220AF
:10061000622062208030A100C03021201430A4006C
:100620005F305A20822B0B30BD000130A2003D0804
:100630000B20A101B61D2B2B3B3041020318222BAE
:10064000C10A2A2BC101173045020318292BC50AFC
:100650002A2BC5012F2B4208C1004608C500051BE7
:100660003F2B4508031D372B0C30C7003E2B0D30A8
:100670004502031C3E2B0C304502C700442B4508A5
:10068000C7002030622062200A30470203184A2B3C
:10069000203062208030A100470828203A306220B4
:1006A0000230A400410829203A3062203030622014
:1006B0006220051B6B2B0C3045020318642B613044
:1006C00062206D306220682B703062206D306220B5
:1006D0001130BD006D2B1330BD00410803190130EE
:1006E000031D0301B5001E30410203190130031D33
:1006F00003013504B50001308618030135040319E0
:10070000822B822D361E802DEB210130C9000F3047
:10071000490203188E2BEB21C90F872B3611B61116
:10072000EB21EB21EB21B61C972B0514982B051020
:100730001230C900143049020318A12BEB21C90F54
:100740009A2BEB210730BC00AF214308C200EB21FC
:10075000361DAB2BB6150630BC00AF214308C600D2
:10076000EB21361DB42BB6150630BC00AF21430873
:10077000BE000330BC00AF214308C8000530BC00F8
:10078000AF214308C0000830BC00AF214308BF00C0
:10079000EB21361DCC2BB615361CD22BB619D12B1E
:1007A00036100120B6197F2D8030A1008030212025
:1007B0000930A40020305A208030A100C030212010
:1007C0001430A40020305A2080302120A1010130B3
:1007D0004802031DF92B4D306220613062206220F7
:1007E0006E306220643062206130622067306220A7
:1007F000702C02304802031D0C2C443062206930FA
:1008000062206E306220733062206430622061307A
:10081000622067306220702C03304802031D212CB7
:10082000573062206F306220653062206E30622067
:100830007330622064306220613062206730622051
:10084000702C04304802031D382C443062206F3075
:1008500062206E3062206430622065306220723027
:100860006220643062206130622067306220702C28
:1008700005304802031D4B2C563062207230622036
:10088000693062206A306220643062206130622008
:1008900067306220702C06304802031D602C5A30ED
:1008A00062206130622074306220653062207230D4
:1008B0006220643062206130622067306220702CD8
:1008C00007304802031D702C5A3062206F306220BE
:1008D0006E306220643062206130622067306220B6
:1008E0008030A100C03021203E0828202030622026
:1008F00001304002031D8B2C6A306220613062207F
:100900006E30622075306220613062207230622069
:10091000693062204A2D02304002031DA02C66304F
:100920006220653062206230622072306220753051
:1009300062206130622072306220693062204A2D6C
:1009400003304002031DAE2C6D3062206130622006
:10095000622072306220743062204A2D04304002DE
:10096000031DBD2C61306220703062207230622025
:10097000693062206C3062204A2D05304002031D30
:10098000C82C6D30622065306220693062204A2DAB
:1009900006304002031DD52C6A306220753062207B
:1009A0006E306220693062204A2D07304002031DFC
:1009B000E22C6A306220753062206C30622069302F
:1009C00062204A2D08304002031DF72C613062205E
:1009D000753062206730622075306220733062208B
:1009E0007430622075306220733062204A2D0930E5
:1009F0004002031D0E2D733062206530622070307E
:100A0000622074306220653062206D306220623076
:100A1000622065306220723062204A2D0A30400226
:100A2000031D212D6F3062206B30622074306220F4
:100A30006F30622062306220653062207230622046
:100A40004A2D0B304002031D362D6E3062206F3070
:100A5000622076306220653062206D306220623024
:100A6000622065306220723062204A2D0C304002D4
:100A7000031D4A2D6430622065306220633062209D
:100A8000653062206D306220623062206530622005
:100A9000723062202030622032306220303062209A
:100AA0008030A1000230A4003F0829200930400214
:100AB000031D692D1430C9000230A20049080B2023
:100AC000A101051C662D5A306220682D5730622026
:100AD0007F2D1230C9000230A20049080B20A1016D
:100AE000051C792D2A3062205A3062202A3062207B
:100AF0007F2D2A306220573062202A306220812DDB
:100B0000AA2D442A851F892D0512831605128312EA
:100B10008B2D8316051683129B30B82041080319CC
:100B20000130031D0301B5000130861803013504AF
:100B300003199B2D0515851585140130A900F43086
:100B4000B9200511851185100130A9004A30B9205E
:100B5000C40A852B01204730622065306220622064
:100B60006E30622020306220733062206930622053
:100B7000673062206E3062206130622062206C300B
:100B80006220203084006030B220A03084005030D9
:100B9000B220203084003030B1200618B616061C72
:100BA000B61203010618013EB61A013C031DDE2DE4
:100BB000B70A0319B80A0130B820D12D0301B61ABB
:100BC0000130013A0319B612031DB61603010618C7
:100BD000013EB61A013C031DF32DB70A0319B80AEA
:100BE0000130B820E62D03303802DE300319370219
:080BF0000318C12D3614442A3C
:02400E00503F21
:00000001FF
